:020000040000FA
:10000000580E0020F9020000010300000303000065
:1000100005030000070300000903000000000000C2
:100020000000000000000000000000000B030000C2
:100030000D030000000000000F030000110300008A
:100040001303000013030000250800001303000041
:10005000130300000000000013030000A1030000D0
:10006000D507000013030000130300001303000072
:100070001303000013030000130300001303000028
:100080001303000013030000130300001303000018
:100090001303000013030000130300001303000008
:1000A0001303000013030000000000000000000024
:1000B0001303000013030000000000000000000014
:1000C0000000000000000000000000000000000030
:1000D0000000000000000000000000000000000020
:1000E0000000000000000000000000000000000010
:1000F0000000000000000000000000000000000000
:1001000000000000000000000000000000000000EF
:1001100000000000000000000000000000000000DF
:1001200000000000000000000000000000000000CF
:1001300000000000000000000000000000000000BF
:1001400000000000000000000000000000000000AF
:10015000000000000000000000000000000000009F
:10016000000000000000000000000000000000008F
:10017000000000000000000000000000000000007F
:10018000000000000000000000000000000000006F
:10019000000000000000000000000000000000005F
:1001A000000000000000000000000000000000004F
:1001B000000000000000000000000000000000003F
:1001C000000000000000000000000000000000002F
:1001D000000000000000000000000000000000001F
:1001E000000000000000000000000000000000000F
:1001F00000000000000000000000000000000000FF
:10020000DFF80CD000F0BAF800480047A10C00005D
:10021000580E002030B4044654E8000F0D4644E860
:100220000053002BF8D1156030BC704730B4044641
:1002300054E8000F40EA010544E80053002BF7D1D1
:10024000156030BC704730B4044654E8000F00EA33
:10025000010544E80053002BF7D1156030BC70470E
:1002600030B4044654E8000F80EA010544E8005326
:10027000002BF7D1156030BC704730B4044654E809
:10028000000F00EB010544E80053002BF7D1156087
:1002900030BC704730B4044654E8000FA0EB0105B1
:1002A00044E80053002BF7D1156030BC704770B4A0
:1002B00004464FF0000054E8006F0D68AE4207BFDF
:1002C00044E80023012044E800630E60002B1CBFBB
:1002D0000020F0E770BC704730B4044654E8000FCB
:1002E00088422CBF451A054644E80053002BF5D13F
:1002F000156030BC7047000006488047064800473C
:10030000FEE7FEE7FEE7FEE7FEE7FEE7FEE7FEE7C5
:10031000FEE7FEE7E9040000010200000048704724
:100320005429000040EA01039B0703D009E008C9F3
:10033000121F08C0042AFAD203E011F8013B00F8AA
:10034000013B521EF9D27047D2B201E000F8012BF6
:10035000491EFBD270470022F6E710B513460A4645
:1003600004461946FFF7F0FF204610BD421C10F866
:10037000011B0029FBD1801A70470000064C074D75
:1003800006E0E06840F0010394E807009847103465
:10039000AC42F6D3FFF738FFC02D0000E02D00007F
:1003A0002DE9FE434FF48278404601F069FA4C4F44
:1003B00000254C4C012600B3404601F069FA94F840
:1003C0002E0010B194F82F10D1B18DF80050616853
:1003D00001912189ADF80810E26832B1218B618367
:1003E00062602181E56010B102E0257400E03E60AA
:1003F00021686846884784F82F5094F82E0060B32F
:100400004FF48077384601F03BFA30B3384601F0BC
:100410003FFA628B94F82D108A420AD9A2EB0100B0
:1004200080B260832289A2EB0000626802EB400088
:1004300005E007D1E06828B184F82F60658301F0FA
:100440000DFA04E08A4202D184F82F6065834046A9
:1004500001F01EFA2248001D06604FF488773846E6
:1004600001F00EFA48B1384601F012FA2574022064
:100470008DF800002168684688474FF48A7738462F
:1004800001F0FEF928B1384601F002FA2574BDE802
:10049000FE834FF000484FF48C7967691DE000BF80
:1004A000B7FA87F028FA00F109EB80058F43284658
:1004B00001F0E6F988B1284601F0EAF9A5F58C7556
:1004C000E8088DF8040045F38000401C8DF80060BA
:1004D0008DF80500216868468847002FE0D1D6E7EF
:1004E00000700040C8000020F0B5A848A74B0126C6
:1004F00000781B1D1A1D4FF0805106280BD11C7867
:10050000240708D11478C4F30314032C06D0042C58
:1005100004D0052C02D0062807D011E0B1F82443FE
:100520009B4DC4F304242C6002E01C78240707D1FF
:100530001478C4F30314032C02D1974D954C6C67C7
:10054000D1F83051D1F84442944FC4F342343C6066
:1005500006280CD11C78240709D11478C4F303149D
:10056000032C04D18E4C276827F0807727604FF04A
:1005700080470024C7F80C41C7F81041874F3F1F40
:100580003C60062807D11F783F0704D11778C7F3CE
:100590000317032F02D0062808D01FE0DFF8FCC1A4
:1005A00003270CF1640CCCF8007007E01F783F07BC
:1005B00014D11778C7F30317032F0FD1DFF8E4C165
:1005C0000527CCF80070774F78373E60754F0837B5
:1005D0003C600CF1040C3F27CCF80070724F3F6870
:1005E000DFF8C8C1CCF800706F4F3F1D3F680CF1B9
:1005F000040CCCF800706C4F08373F680CF1040C09
:10060000CCF80070684F0C373F680CF1040CCCF844
:100610000070654F10373F680CF1040CCCF8007087
:10062000614F14373F680CF1040CCCF800705E4F3A
:1006300018373F68DFF874C10CF1200CCCF800705B
:10064000594F1C373F680CF1040CCCF80070564F22
:1006500020373F680CF1040CCCF80070524F24375F
:100660003F680CF1040CCCF800704F4F28373F68FE
:100670000CF1040CCCF800704B4F2C373F680CF198
:10068000040CCCF80070484F30373F68DFF81CC1CD
:100690000CF1400CCCF80070434F34373F680CF13C
:1006A000040CCCF80070404F38373F680CF1040C54
:1006B000CCF800703C4F3C373F680CF1040CCCF890
:1006C0000070394F40373F680CF1040CCCF80070D3
:1006D000DFF8DCC0FB27CCF80070062813D11F78A8
:1006E0003F0710D11778C7F30317032F03D0042F48
:1006F00001D0052F07D1D1F85872DFF8B8C007F044
:100700004F07CCF800702C480268D20702D06FF077
:1007100001020260062D08D1D1F83401062804D167
:100720002648016841F4806101604FF01021D1F842
:100730000002002803DBD1F80402002822DA204A54
:10074000166020480368002BFCD01523C1F8003246
:100750000568002DFCD0C1F8043201680029FCD0E6
:10076000146001680029FCD0BFF34F8F0C48F038AB
:100770000168154A01F4E06111430160BFF34F8F36
:1007800000BFFDE7124911480860F0BDE00F00F01E
:10079000403501400DF0ADBA00C007403C050040B7
:1007A000FCED00E0105600400404001020C500409D
:1007B00018F50040E40E0040000400403C170040E3
:1007C00004E5014000E401400400FA050090D00374
:1007D000940000202DE9F047104E042700244FF428
:1007E000A0784FF4803900BF08EB840509FA04F0C3
:1007F000715961B1D6F80413014208D02946304638
:1008000001F08EF80648D0E9002128469047641C84
:10081000E4B2BC42E8D3BDE8F087000000800040AD
:10082000F80000200149024801F00EBE040100203A
:100830000020004002E008C8121F08C1002AFAD1B7
:1008400070477047002001E001C1121F002AFBD150
:100850007047000072B600F00FFF00BF00F04AFDC5
:100860000028FBD1104C0121208801EB00400FA192
:1008700000F04CFE10480068C00700D000BE208881
:10088000022101EB00400DA100F040FEBFF34F8FAD
:100890000948E43801680D4A01F4E0611143016040
:1008A000BFF34F8F00BFFDE7B000002046617461C9
:1008B0006C206572726F7200F0ED00E05379737412
:1008C000656D207265736574000000000400FA0510
:1008D0000EB500210091CDE901106A4644F20100F5
:1008E000FFF7B8FF0EBD00F003B800F009B8000034
:1008F00072B602480168491C016070471C00002064
:1009000003490868401E086000D162B670470000C5
:100910001C0000202DE9F041064608680C46411CE9
:100920004FF0A0474FF0010506D005FA00F1C7F8D7
:100930000815206800F006FC6068411C02D0002108
:1009400000F0F7FB3168A069C1F82405607D217DC6
:1009500032680843C2F86C05D4E900123068C0F868
:100960000C15C0F81425207D012815D1A068411C64
:1009700002D0002100F0DDFBE068411C05D085407D
:10098000C7F80855E06800F0DDFBD4E902123068D2
:10099000C0F80825C0F81015BDE8F0812DE9F04732
:1009A0000546861C90460F464FF001090020FFF7D0
:1009B0009AFF1B4C20683860D4E90001401AA168F6
:1009C00004F21C47081A0EE00121384600F0FCF939
:1009D00000F018F90146384600F0F6F9D4E90001B4
:1009E000401AA168081A401C8642EDD8B8F1000FE1
:1009F00003D0052065F3891002E0062065F39F50BF
:100A0000A2682168114004EB8101C860206830446D
:100A100020600020FFF769FF4846BDE8F08700002E
:100A20003402002030B482680468531C8360A154EF
:100A3000D0E901128A4202D330BC00F066BA30BC61
:100A400070470000034803C8814201D1012070476C
:100A5000002070473402002010B50021024800F049
:100A6000BEF980F3100010BD500600202DE9FC5F98
:100A70000E008346DDE90C47C6F100009846924619
:100A8000814600D40846012503E000BF90FBFAF040
:100A90006D1C5045FADAA84500D9454624B1002E10
:100AA00001DB780700D5641EB80702D5B8F1000F46
:100AB0000AD0F80708D13CB1A54205D220215846FA
:100AC000641EFFF7AFFFF6E7002E02DA4E462D2137
:100AD00002E0780703D52B215846FFF7A3FF07F064
:100AE000030002280BD1B8F1000F08D13CB1A54298
:100AF00005D230215846641EFFF794FFF6E7CDE992
:100B00000047434652463146584601F017FDBDE8BE
:100B1000FC9F000070B50D46044600684FF48871D4
:100B200000F009FF4FF49071206800F004FF4FF4CB
:100B30009271206800F0FFFE4FF4A271206800F06F
:100B4000FAFE20681249C0F8041320686907000BF8
:100B500040B2090E002806DA00F00F0000F1E02094
:100B600080F8141D03E000F1E02080F800142068F4
:100B70000121000B40B200F01F02914040098000AB
:100B800000F1E020C0F88012C0F8001170BD000034
:100B900010030200024600201268930702D0530798
:100BA00002D47047500714D502F00300012802D088
:100BB00002280CD105E0C2F383100B68801C184496
:100BC00004E00223086803EB9252104408600120FD
:100BD0007047086800EB9253C2F38910401CEEE79F
:100BE0000121814003484068014201D00120704743
:100BF000002070471400002001218140080300D02C
:100C0000012070472DE9FF410026234800F0D9F864
:100C10002148001F074600F0D4F8204C606800907F
:100C2000A56800E000986946284004EB80000C307D
:100C3000FFF7B0FF0028F5D101AA009901EA0503EA
:100C400004EB8303491CDB6842F82030401C009110
:100C50000228F2D3019800F0030001280BD00228EB
:100C600010D10198032101EB90500099BDF80A6062
:100C700001EB900005E00198BDF80A60C0F3831015
:100C800008440090384600F099F808B10098606078
:100C900004B03046BDE8F0814C060020340200204C
:100CA0004FF40041002000F0A3FC08B1FFF710FE54
:100CB00000F012FB00F0BAFD08B1FFF709FE01F0E9
:100CC0009DFA01F0D5FA01F0C5FA08480321008821
:100CD00001EB004006A100F019FC00BF00F0BAFDD6
:100CE00000F008FB0028FBD1F8E70000B00000206E
:100CF00053414144432048414C2073696D706C65F9
:100D0000206578616D706C652073746172746564C0
:100D10002E0000002DE9F047C7880446181D16462E
:100D20008946B0FBF7F1B0FBF7F207FB12009A1906
:100D30003A44D21CB2FBF7F2DDF820A001E02468AF
:100D4000491E0029FBD13D1A8846B54216D818E045
:100D5000BAF1000F05D0211809EB08002A46091D39
:100D600004E0204409EB08012A46001DFFF7DAFAE7
:100D700000202468761BA844B74201D9354600E01C
:100D80003D46002EE4D1BDE8F087000030B50246B4
:100D900059B100F059FC0021074C09E004EB810334
:100DA00015685B88AB4202D11160002030BD491C40
:100DB0008142F3D3052030BD98000020002100F0CF
:100DC00009B8012100F010B808B56A46FFF755FAD6
:100DD000009808BD08B56A46FFF735FA08BD08B5A2
:100DE0006A46FFF717FA08BD08B56A46FFF71EFA0C
:100DF000009808BD08B56A46FFF74CFA009808BD90
:100E000070B5044600252846FFF76DFD216862682D
:100E1000086890420ED9401E08600178A38AE268F3
:100E200001FB0325227A2168101AC0B20A79824296
:100E300000D208710020FFF758FD284670BD70B53C
:100E400005460C460020FFF74EFDE868A98A201AE7
:100E5000B0FBF1F12A681068431C13600170BDE813
:100E600070400020FFF741BD10B530B1017A4268F3
:100E70000368891AC9B21A6006E00E2010BD036823
:100E80001A68541C1C601170491EC9B2F7D2006860
:100E900000210171084610BD0448017809B1852080
:100EA00070470121017000207047000008000020F9
:100EB00070B5064604780C4888B0154640F82420E2
:100EC000094A0869121D42F8240020226846FFF7EB
:100ED00029FA04940DB1054A00E000226946301D4C
:100EE00000F0F2FF08B070BD0C00002019240000D3
:100EF0000FB408B50399002904D004AA00926A46E9
:100F000000F00FF801B05DF814FB10B582680446DC
:100F1000002A05D0D4E90403216898470020A06086
:100F200010BD2DE9FC4791460C00804676D014F8A0
:100F3000011B39B125290ED04046FFF773FD2078FB
:100F40000028F4D198F80C00002867D04046BDE88E
:100F5000FC47FFF7DABF0020012221782B291BD0A4
:100F60002D2902D0302908D102E040F0010001E033
:100F700040F00200641C002AEFD100252A290ED07F
:100F80002178A1F130020A2A11D205EB850201EB8A
:100F90004205641C303DF1E740F00400EAE7D9F86F
:100FA00000100B1DC9F800300968641C0D4421783D
:100FB00000232E290BD114F8011FA1F130020A2AB7
:100FC00005D203EB830201EB4203303BF3E76C29CC
:100FD0000DD068290BD0692921D00BDC252918D028
:100FE000582931D063290ED0642915D117E014F89F
:100FF000011FECE7702969D0732932D075291BD005
:10100000782909D120E0D9F80000011DC9F80010A5
:1010100001784046FFF706FD641C90E76CE0D9F8C4
:1010200000100A1DC9F800200968CDE900500A2205
:101030004046FFF71BFDEFE7D9F800100A1DC9F87D
:10104000002009680A2206E0D9F800100A1DC9F834
:10105000002009681022CDE90050404601F06EFAE8
:10106000DAE7D9F8001000270A1DC9F800200E6839
:10107000C00705D112E04046761C7F1CFFF7D2FC6A
:1010800031780029F7D104E0202140466D1EFFF79A
:10109000C9FCBD42C0D9002DF6D1BDE74EB13046E6
:1010A000FFF764F9074604E0202140466D1EFFF774
:1010B000B9FCBD4206D9002DF6D103E04046761CAE
:1010C000FFF7B0FC31780029F8D1A5E7D9F8000086
:1010D000011DC9F80010056830214046FFF7A2FC49
:1010E00078214046FFF79EFC08200021CDE9000151
:1010F000034610222946B0E7BDE8FC8770B541EAF7
:101100004201DDE904564FF0A04441EA830141EA7F
:10111000052104EB800041EA0641C0F8001770BDCC
:101120001CB5002100910B4601220191FFF7E6FF5B
:101130001CBD1CB500220B46009211460192FFF720
:10114000DDFF1CBD1CB5002100910B460122019161
:101150001146FFF7D3FF1CBD30B5124B01460020EE
:10116000D3F81044224609E0157A854205D1401C87
:101170000A28F7DB4FF0FF3030BD5268002AF3D168
:10118000421CF9D00872D3F810242AB152684A6080
:10119000D3F81024516030BD0022C3F810144A6007
:1011A00030BD000034020020F0B595B01C46154655
:1011B0000F4608461A9E00F017FB182109A8FFF7F2
:1011C000CAF80E96CDE909540023082203A938462F
:1011D00000F01FFB05980690BDF81000ADF81C004C
:1011E000BDF81200ADF81E0000208DF82100039814
:1011F000082600F00300012802D0022818D032E0AF
:1012000003983346850AC0F3C2008DF82000039886
:101210000FA9C0F38314A200384600F0FAFA09A817
:10122000009006AB22460FA9284600F039FA1AE0D2
:101230000398840DC0F3C2008DF82000082C01D261
:10124000254600E0082533462A460FA9384600F017
:10125000E0FA2E44641B09AB06AA29460FA800F049
:1012600071F9002CEAD1384600F0C4FA15B0F0BD8F
:101270007047012001F0A8B810B5044800F0B0FE96
:10128000BDE81040002001F09FB8000030000020B1
:1012900008B5034A00924023024AFFF785FF08BDC4
:1012A00001230000340100200A4A012902EBC0009A
:1012B00007D0022907D0032907D0042907D000202E
:1012C00070470220704704207047007970474079CA
:1012D00070470000E02D000010B5FFF7CAFF0421A1
:1012E0000348FFF739FF02490120487210BD000092
:1012F000380000202DE9F0478CB0FFF7A3FB18B1B0
:1013000000200CB0BDE8F087784C0020C4F8180429
:10131000BFF34F8F60680290A5684FF00008284027
:1013200004EB800008E021680298814201D86160E6
:10133000E6E7284004EB80000C3002A9FFF72AFC06
:101340000028F0D103AB029901EA050204EB820206
:10135000491CD26843F82020401C02910228F2D395
:10136000039800F00300022802D001284ED0A5E027
:1013700003985022810D8946B2EB905F00D850212E
:101380000E4666F39F5003900831594800F0E3F988
:10139000070078D000F028FA4346082203A938460F
:1013A00000F03DFA029908F1080A2940681A800005
:1013B000001D864223D94D4D0C3530B1C2B204EB2D
:1013C0008101301A90460C3104E02946F2B2002522
:1013D00090462846C6B25346384600F020FA0AEB3B
:1013E00008032DB1324629464FEA070000F017FAEC
:1013F000029909F1030001EB900002903AE004EB3E
:1014000081015346324638460C31EFE70398C0F36A
:101410008311062900D3062161F389100390C0F3DC
:101420008310801C8100324800F095F9070045D0F8
:1014300000F0DAF94346082203A9384600F0EFF934
:1014400008F1080800260FE00298434600EA05016B
:10145000401C04EB81010290042238460C3100F05C
:10146000DEF908F10408761C0398C0F38310B0423B
:10147000EAD847B1D4F81054D4F8180468B1384603
:1014800000F0B8F92CE019E0687A012804D12A6844
:1014900028463946126890476D68002DF4D13846C9
:1014A00000F0A8F90020FFF71EFAD4F8180408B9D4
:1014B000029860600020FFF718FA11E0D4F8104499
:1014C00004E021682046896888476468002CF8D1C8
:1014D00008480221008801EB004007A100F016F83F
:1014E000FFF7B0FA80F001000BE7000034020020A3
:1014F000182E0000B00000204261636B656E6473BB
:1015000020666C75736865640000000000231A464D
:1015100000F00CBF08B5012300926A4600F006FFF8
:1015200008BD1CB5CDE9002302236A4600F0FEFE8B
:101530001CBD3EB5069C8DE81C0003236A4600F0E6
:10154000F5FE3EBD2DE9F0470E4680461C4692460C
:1015500008293ED894F80C900020207319461046B4
:1015600000F0B4FD0025B54206D218F805201AA1F6
:101570002046FFF7BDFC03E019A12046FFF7B8FCA9
:101580006D1C082DEFD317A12046FFF7B1FC0025F5
:10159000B54210D218F80570FEF7C0FE0068C05DB5
:1015A00010F03E0F01D03A4600E02E220EA1204658
:1015B000FFF79EFC03E00DA12046FFF799FC6D1C90
:1015C000082DE5D301222146504600F061FD84F844
:1015D0000C90BDE8F0870000202530327800000034
:1015E000202020007C000000256300002000000077
:1015F000104810B5FF218160002101604160C0F8F2
:101600001814C0F8141480F820140B4800F0F0F8F7
:1016100000280DD109480A490A4B401AC108002088
:1016200003E000BF23F82000401C8842FAD30020CA
:1016300010BD000034020020182E0000182E0000FB
:10164000E02D00009800002002480349401AC0081D
:1016500070470000182E0000E02D000013B568460A
:10166000FFF794FB08B100201CBD0248009950F818
:1016700031001CBDE02D000070B508480125D0F8F0
:10168000104480F8205405E06572216820464968BE
:1016900088476468002CF7D170BD00003402002038
:1016A0002DE9FF4781460C9D00200C462F7B2873B7
:1016B000984616462946184600F008FD072E42D2E5
:1016C000DFE806F004090F161F2A360049462846AF
:1016D000FFF70EFC37E0494628462268FFF708FC72
:1016E00031E0D4E9002349462846FFF701FC2AE00F
:1016F000A0680090D4E9002349462846FFF7F8FB8C
:1017000021E0D4E90201CDE90001D4E900234946F2
:101710002846FFF7EDFB16E004F1080007C88DE846
:101720000700D4E9002349462846FFF7E1FB0AE019
:1017300004F108000FC88DE80F00D4E900234946E2
:101740002846FFF7D5FB00222946404600F0A0FCC2
:101750002F73BDE8FF872DE9F041858A80462D1F54
:101760004819C01CB0FBF5F0C6B24046FFF748FB75
:10177000041E19D00020207101206071E58000272F
:101780002546761EC4F800800BE04046FFF738FB84
:1017900060B16179491C6171286005467F1CC0F801
:1017A0000080B742F1D32046BDE8F081204600F02A
:1017B00002F80020F8E72DE9F041457901466B1E5B
:1017C000002201E00968521C9A42FBD30F680146CF
:1017D000002605E038460C68FFF731FB2146761CF1
:1017E000AE42F7D3BDE8F0810121001DFFF7ECBA4E
:1017F000FFF73ABB10B504460121001DFFF7FAFAC6
:1018000010F0FF0F04D12046BDE81040FFF7D3BF12
:1018100010BD38B501240094FFF77CFA38BD38B507
:1018200000240094FFF776FA38BD0000064910B591
:1018300000204870091D0860BFF35F8F034904480A
:1018400000F030F8002010BD200000206C270000C0
:101850002801002020BF40BF20BF7047024A10600F
:10186000101D0160704700002C7600400301034802
:101870001844C0F81425C0F81015704700700040D7
:1018800002494058002800D00120704700700040F5
:10189000034908B50844002202600068009008BDB2
:1018A00000700040016009684160AFF3008010B52E
:1018B000D0E900215368994201D1002104E0D1E927
:1018C0000034A34202D01946816010BD0831416046
:1018D000F0E700000C4A10B502F58C730EE0991A7F
:1018E000C91001EBD171491002EBC1010C688442AF
:1018F00001D90B4602E005D201F108029A42EED36B
:10190000002010BD486810BD8C27000000B5FFF70F
:10191000E1FF002800D1014800BD00007827000049
:1019200008B5002242504058009008BD4058002899
:1019300000D00120704708B5002242504058009066
:1019400008BD0121B1EB507F01D10120704700207B
:10195000704700002DE9F05F0427204EDFF88090EB
:10196000834600244FF0030A4FF001080020FEF7E1
:10197000BAFF08FA04F5354203D02046FFF730F9E4
:10198000B8B10020FEF7B1FFFFB104F10104AE438E
:10199000E4B2EBD13846FFF7B9FFB9F800100346BF
:1019A0000AEB01400F4A10A1FFF7BBFD3846BDE826
:1019B000F09F154908FA04F000274A681043486070
:1019C0008BF800403846FEF790FFB9F80010224629
:1019D0000AEB01400DA1FFF79DFDDBE7FFFF0F00C4
:1019E000B00000200D26000046756E6374696F6EAE
:1019F0003A2025732C206572726F7220636F6465C4
:101A00003A2025732E00000014000020416C6C6FFA
:101A10006361746564206368616E6E656C3A20254D
:101A2000642E00002DE9F84314460D0081462CD0A9
:101A3000002C2AD00026FFF7DFF8174F4FF00308DD
:101A4000002824D04846FFF7CBF8002821D01348BF
:101A500000EBC900C0F81055C0F81445009439884F
:101A60002B4608EB01404A460DA1FFF762FD3046C8
:101A7000FFF74CFF3988034608EB0140184A19A1CB
:101A8000FFF74FFD3046BDE8F8830E20FBE7072641
:101A9000EDE70826EBE70000B000002000F0014071
:101AA00041737369676E6564206368616E6E656C0F
:101AB0003A2025642C206576656E7420656E64205E
:101AC000706F696E743A2025782C207461736B20D6
:101AD000656E6420706F696E743A2025782E000060
:101AE0003A26000046756E6374696F6E3A2025735E
:101AF0002C206572726F7220636F64653A202573C3
:101B00002E00000070B5044601260025A640FFF710
:101B100073F818B12046FFF763F880B109480660F2
:101B20002846FFF7F3FE034607480321074A0088CB
:101B300001EB004006A1FFF7F4FC284670BD082524
:101B4000EEE7000004F50140B00000206F26000021
:101B500046756E6374696F6E3A2025732C2065722A
:101B6000726F7220636F64653A2025732E00000047
:101B700000207047704700002DE9F041254C0646D3
:101B800012200D46C4F808032348017C022918D00E
:101B9000027C01464FF4807891F82E10012A12D071
:101BA0000222C4F80423012707744660058100223D
:101BB000C26021B3458390F82D103046FFF74EFEEA
:101BC00025E0122002E0C2682AB10220C4F8040312
:101BD0001120BDE8F081C660058361B947463846EB
:101BE000FFF74EFE0028FAD03846FFF751FE29468F
:101BF0003046FFF733FE0220C4F8040307E029460D
:101C00003046FFF72BFE4046FFF742FE27600020DC
:101C1000DFE7000000700040C800002070B50546F6
:101C20002A480C46017C09B1112070BD2179284E4B
:101C300009B1012901D10021316000EB45010A7F82
:101C40001AB910F82D2F521C0270E0790877207A0B
:101C5000487721786278302301F0030103EA021209
:101C60001143A2784FF4E06303EA02221143E278C1
:101C70004FF4805303EA0232114322794FF4E023F8
:101C800003EA0242114362794FF4801303EA0252DD
:101C90001143A2791B0103EA02620E4B284611434D
:101CA00003EB0012C2F81815227AE179FFF7DEFD86
:101CB000227AE1792846FFF7D9FD207908B1012879
:101CC00001D101203060002070BD0000C80000205C
:101CD00000750040007000402DE9F0411E4C0546A3
:101CE00094F82C0010B10820BDE8F08144F8101BD6
:101CF0001A4928780860091D68780860E878A07794
:101D0000012727770020207060776060144EE0770D
:101D10006FF00040C6F808034FF48270FFF7B8FD7B
:101D2000B015FFF7B5FDA8780E49400181F8000411
:101D30008020C91FC1F88002C1F800010220C6F846
:101D40000403A07F10B10120C6F804030348F03853
:101D500007600020C8E70000C8000020F0750040C0
:101D60000070004007E000E0044890F82E0008B141
:101D7000002000E00420024908447047C800002009
:101D8000007000402DE9F04106460D464FF48034C6
:101D900000681746AC404BB14FF4A07101EB8501D0
:101DA000FFF7BEFD3068C0F8044301E0C0F8084307
:101DB000306800EB8500C0F84075BDE8F081000098
:101DC000016801220A600079034A00EB400002EB3F
:101DD0008000022101727047F8000020F0B404680E
:101DE000049E40F20115D4F800728D40AF43C4F850
:101DF00000720468D4F800521D43C4F80052334600
:101E0000F0BCFFF7BFBF00002DE9F04104460E46CD
:101E100000792C4900EB400001EB8007387A10B1C3
:101E20000820BDE8F0813A60706800254FF4A07882
:101E3000786006E008EB85012068FFF771FD6D1CF6
:101E4000EDB26079A842F5D82068F178000B40B275
:101E500000284FEA411106DA00F00F0000F1E020FF
:101E600080F8141D03E000F1E02080F800142068E1
:101E70000122000B40B200F01F0302FA03F14009F7
:101E8000800000F1E020C0F88012C0F80011206846
:101E90007178D0F8043561F30103C0F80435206887
:101EA000B178D0F8083561F30103C0F8083520682F
:101EB0003178D0F8103561F30303C0F810353A7269
:101EC0000020AEE7F80000202DE9F0410546164657
:101ED00000790F46154A00EBC00102EB810494F82B
:101EE000201011B10820BDE8F081114951F82010EF
:101EF0002868FFF73DFE08B11120F4E7394628466F
:101F0000FEF708FD6660386920601EB1397F2846FB
:101F1000FEF700FE28680821C0F800150020A06127
:101F2000E0610121606184F82010DCE704010020F9
:101F3000402700002DE9F04704460E46007920496D
:101F400000EBC00001EB800517463046FFF7F9FCB7
:101F500030B1204600F036F820B11120BDE8F087FE
:101F60001020FBE76F61AE604FF49076002731469A
:101F70002068FFF7E0FC4FF4AC7841462068FFF79B
:101F8000DAFC2068AA686969C0F84425C0F84815D9
:101F9000206801218160686878B9B14649462068A7
:101FA000FFF7C4FC064641462068FFF7BFFC064326
:101FB000F4D000B10F27002068613846CEE700005A
:101FC000040100200079054900EBC00001EB80000E
:101FD0004069002800D00120704700000401002063
:101FE0002DE9F04704460079274900EBC00001EBDA
:101FF000800720684FF00009C0F80095786880B12C
:1020000020682249C0F8081320680121000B40B263
:1020100000F01F0291404009800000F1E020C0F86C
:1020200080112068D0F80C25D0F81485D0F8086508
:10203000D0F810554FF0FF31C0F80C15C0F814154A
:102040002068C0F80815C0F81015501C02D01046C2
:10205000FFF766F8B8F1FF3F02D04046FFF760F89F
:10206000681C02D02846FFF75BF8701C02D030468F
:10207000FFF756F82068FFF77DFD87F82090C7F836
:102080000490BDE8F0870000040100201003020066
:1020900010B50C46017A052908D0407A38B10848B5
:1020A00008A102682046FEF723FF00E01AB106A14E
:1020B0002046FEF71DFF2046BDE81040FEF725BF75
:1020C00070000020257300000D0A000038B5C38899
:1020D0000D46044633B114A0009015A216A128465F
:1020E000FEF706FF217A05291CD0607A48B1A08846
:1020F000FFF7DAF8164951F8202016A12846FEF716
:10210000F7FEA0880021FFF7A9FA03461049207ABC
:10211000143951F8202001B02846BDE830400EA106
:10212000FEF7E6BE38BD00001B5B306D000000000E
:102130001B5B313B33316D0025734C6F677320643B
:10214000726F70706564202825642925730D0A005C
:1021500070000020257300003C25733E2025733A53
:10216000200000001FB501238DF800308DF8081005
:102170000192D0E90012684690471FBD2DE9F04159
:1021800005460078002824D105216868FFF7F4FC93
:1021900008B1FEF79DFB104FDFF84080032638881A
:1021A0000FA106EB0040D8F80420FFF7B3F9002494
:1021B000686811A130F91420388806EB0040FFF759
:1021C000A9F9641C052CF3DBD8F80410491CC8F8E5
:1021D0000410BDE8F0810000B000002000000020E5
:1021E000414443206576656E74206E756D6265723C
:1021F0003A20256400000000256400000EB5124A54
:1022000007CA8DE80700104810491438FFF764FD2D
:1022100008B1FEF75DFB69460020FFF7FFFC08B13F
:10222000FEF756FB05210A48FFF7A6FC08B1FEF7AA
:102230004FFB074805210A30FFF79EFC002801D01C
:10224000FEF746FB0EBD0000042600007D210000C5
:10225000B4000020054810B50078FFF753FC0028B3
:1022600003D0BDE81040FEF733BB10BD00000020D6
:102270003EB5FEF711FE08B1FEF72AFB1C491D4AC8
:10228000D1E90301CDE9010103208DF806001848CA
:1022900001A9001DFFF7B8FD08B1FEF719FB144CAA
:1022A000241D2068D0F81005134A0123C2400020E5
:1022B000014600902046FFF791FD2046FFF780FD84
:1022C000246804F5A074FFF74FFD05460B48FFF79F
:1022D00041FB08B1FEF7FCFA08482A46214600787F
:1022E000FFF7A0FB002801D0FEF7F2FA3EBD000088
:1022F000F0250000B923000000A8610000000020C4
:1023000010B5094C0020D2B2207004F10800FFF78C
:1023100011FE08B1FEF7DCFA6078002802D02178BF
:102320000029FAD010BD0000280000202DE9F84F48
:10233000204D92468946064698460122694618462F
:10234000AF68FEF72BFB58B3009800210446801CB1
:1023500009E000BF00EA07035AF8212005EB8303D8
:10236000401C491CDA604145F4D34FEA164AFEF797
:1023700073FB4AEA0041601C384005EB80003C409A
:1023800005EB8402C160D06866F3C50068F389106C
:1023900069F39F2020F00300401C20F00400D0606F
:1023A00095F8200402E000BFFEF7A4FF0028FBD14F
:1023B000BDE8F88F34020020704700000149012079
:1023C000087070472800002010B588B0044620220D
:1023D0000E496846FDF7A6FF06200090C01F019039
:1023E000029003904FF0EB7006900CB1084A00E0A9
:1023F000002269460748FEF75BFD08B1FEF768FA60
:102400000448001F447008B010BD0000B028000050
:10241000BD2300002C0000201FB50A4601788DF86E
:10242000001041680191017A8DF80810C06803908E
:10243000044850F82210001F50F8222068469047A8
:102440001FBD0000100000202DE9FF410C464FF495
:10245000927705463946FFF769FA0026C0B139463A
:102460002846FFF768FA02208DF80000D5F88004AE
:10247000C5F880040390D5F83C058DF80800E068A5
:102480000190A661E661D4E900126846904723E016
:102490004FF4887739462846FFF748FAE0B13946C5
:1024A0002846FFF748FAD5F83C15A069884213D1B1
:1024B000E06960B1E268D5F8000220F02000C5F8BC
:1024C0000002E069A0612069E661E06001E0A661C8
:1024D000E2682046FFF746FE4FF4A27739462846C9
:1024E000FFF724FA60B139462846FFF724FAA069BD
:1024F00030B1A661D5F83C152046E268FFF732FE00
:102500004FF4907739462846FFF710FA002813D089
:1025100039462846FFF70FFA606900280CD0D5F835
:102520004C058DF800608DF80800A0680190666188
:10253000D4E9001268469047BDE8FF812DE9F05FBD
:102540008346DDE90A4A994690460D46084601272A
:1025500003E000BFB0FBF8F07F1C4045FAD2B9455C
:1025600000D94F465FEACA7012D18CB15FEA8A7017
:1025700002D5B9F1000F01D0202607E0302605E092
:1025800031465846641EFEF74DFA0CB1A742F7D308
:102590005FF00106B9F1010F02D9A9F1010903E0C9
:1025A000B5FBF6F0404502D306FB08F6F2E7DFF88C
:1025B0003C9000BFB5FBF6F000FB165519F8001073
:1025C0005846FEF72FFAB6FBF8F6002EF2D15FEA76
:1025D000CA7009D0002C07D0A74205D22021584646
:1025E000641EFEF71FFAF5E7BDE8F09F44270000E0
:1025F0000100070000800040000400000000000708
:10260000000000000000000002000001006E726681
:10261000785F7070695F6368616E6E656C5F616C36
:102620006C6F63006E7266785F7070695F6368617B
:102630006E6E656C5F66726565006E7266785F705F
:1026400070695F6368616E6E656C5F617373696703
:102650006E006E7266785F7070695F6368616E6E3F
:10266000656C5F666F726B5F61737369676E006E36
:102670007266785F7070695F6368616E6E656C5FCB
:10268000656E61626C65006E7266785F7070695F1E
:102690006368616E6E656C5F64697361626C65002E
:1026A0006E7266785F7070695F67726F75705F6178
:1026B0006C6C6F63006E7266785F7070695F6772D2
:1026C0006F75705F66726565006E7266785F7070B8
:1026D000695F67726F75705F656E61626C65006ED1
:1026E0007266785F7070695F67726F75705F64693A
:1026F0007361626C65006E7266785F7070695F63AB
:1027000068616E6E656C735F72656D6F76655F662E
:10271000726F6D5F67726F7570006E7266785F7052
:1027200070695F6368616E6E656C735F696E636C20
:102730007564655F696E5F67726F75700000000099
:1027400025080000303132333435363738394142CC
:102750004344454600000000000000000000000067
:1027600000000000000000000000000054270000EE
:102770006C27000004000000556E6B6E6F776E20B2
:102780006572726F7220636F646500000000000064
:10279000BC2C0000010000007C2B000002000000A7
:1027A0007029000003000000F02B0000040000006E
:1027B000442C000005000000242B0000060000004F
:1027C000C02A0000070000002C2C000008000000B8
:1027D000382B0000090000009C2B00000A000000BC
:1027E000A42C00000B000000582900000C00000081
:1027F000502B00000D000000F42C00000E00000023
:102800001C2C00000F000000582C000010000000DD
:102810008C2C000011000000082D0000800000003A
:10282000D82A000081000000142A00008200000065
:10283000D429000083000000B429000084000000B7
:10284000F029000085000000FC2A0000860000003E
:10285000042C000090000000A02A0000910000005D
:102860009429000092000000642B00000082000008
:102870006C2C000001820000B82B000002820000D6
:10288000D42B000000840000302A000001840000E6
:10289000C82C000002840000782A00000384000095
:1028A000542A0000911200007912000071120000F9
:1028B000FFFFFFFFFFFFFFFFFFFFFFFFFFFFFFFF28
:1028C00000000000000000000000D601070000002A
:1028D0000040404040404040404041414141414033
:1028E00040404040404040404040404040404040E8
:1028F0004005020202020202020202020202020277
:10290000022020202020202020202002020202027B
:1029100002029090909090901010101010101010D3
:1029200010101010101010101010101002020202DF
:102930000202888888888888080808080808080823
:10294000080808080808080808080808020202021F
:1029500040000000D12800004E52465F4552524FC1
:10296000525F494E56414C49445F44415441000036
:102970004E52465F4552524F525F534F4654444564
:10298000564943455F4E4F545F454E41424C454486
:10299000000000004E52465F4552524F525F46457E
:1029A00041545552455F4E4F545F454E41424C4550
:1029B000440000004E52465F4552524F525F4D5503
:1029C0005445585F554E4C4F434B5F4641494C452B
:1029D000440000004E52465F4552524F525F4D55E3
:1029E0005445585F4C4F434B5F4641494C4544006A
:1029F0004E52465F4552524F525F4D555445585FB7
:102A0000434F4E445F494E49545F4641494C45440B
:102A1000000000004E52465F4552524F525F4D55E6
:102A20005445585F494E49545F4641494C4544001E
:102A30004E52465F4552524F525F424C455F49509D
:102A400053505F52585F504B545F5452554E434160
:102A5000544544004E52465F4552524F525F424CDD
:102A6000455F495053505F504545525F52454A4576
:102A700043544544000000004E52465F4552524FB9
:102A8000525F424C455F495053505F4C494E4B5F3B
:102A9000444953434F4E4E454354454400000000C3
:102AA0004E52465F4552524F525F4150495F4E4F22
:102AB000545F494D504C454D454E5445440000002F
:102AC0004E52465F4552524F525F4E4F545F5355E0
:102AD00050504F52544544004E52465F4552524F5B
:102AE000525F4D4F44554C455F4E4F545F494E49E0
:102AF0005449414C495A4544000000004E52465F3B
:102B00004552524F525F4D4F44554C455F414C52D8
:102B1000454144595F494E495449414C495A4544FD
:102B2000000000004E52465F4552524F525F4E4FDA
:102B3000545F464F554E44004E52465F4552524FE9
:102B4000525F494E56414C49445F535441544500ED
:102B50004E52465F4552524F525F444154415F537B
:102B6000495A45004E52465F4552524F525F494FB7
:102B70005F50454E44494E47000000004E52465FAC
:102B80004552524F525F5356435F48414E444C4565
:102B9000525F4D495353494E470000004E52465F25
:102BA0004552524F525F494E56414C49445F4C4545
:102BB0004E475448000000004E52465F4552524F67
:102BC000525F4452565F5457495F4552525F414EDF
:102BD00041434B004E52465F4552524F525F445262
:102BE000565F5457495F4552525F444E41434B0034
:102BF0004E52465F4552524F525F494E5445524ED7
:102C0000414C00004E52465F4552524F525F535462
:102C10004F524147455F46554C4C00004E52465F6F
:102C20004552524F525F4E554C4C00004E52465F3B
:102C30004552524F525F494E56414C49445F5041B4
:102C400052414D004E52465F4552524F525F4E4FD9
:102C50005F4D454D000000004E52465F4552524FB9
:102C6000525F464F5242494444454E004E52465FE1
:102C70004552524F525F4452565F5457495F455236
:102C8000525F4F56455252554E0000004E52465F1D
:102C90004552524F525F494E56414C49445F414460
:102CA000445200004E52465F4552524F525F494EC9
:102CB00056414C49445F464C414753004E52465F93
:102CC00053554343455353004E52465F4552524F6E
:102CD000525F424C455F495053505F4348414E4E0E
:102CE000454C5F414C52454144595F455849535406
:102CF000530000004E52465F4552524F525F5449B6
:102D00004D454F55540000004E52465F4552524FBC
:102D1000525F4255535900007761726E696E6700C9
:102D200064656275670000001B5B313B33306D00EA
:102D30001B5B306D000000001B5B313B33316D00CD
:102D40001B5B313B33326D001B5B313B33336D001A
:102D50001B5B313B33346D001B5B313B33356D0006
:102D60001B5B313B33366D001B5B313B33376D00F2
:102D7000696E666F000000006572726F720000007D
:102D800050525300534141444300000054494D45C3
:102D90005200000055415254450000007077725FA8
:102DA0006D676D740000000062616C6C6F632E6C67
:102DB0006F675F6D656D706F6F6C000061707000A4
:102DC000302E000000000020B40000003408000095
:102DD000E42E0000B4000020A40D00004408000010
:102DE000802D000000000000842D00000000000085
:102DF0008C2D000000000000942D00000000000059
:102E00009C2D000000000000A82D00000000000321
:102E1000BC2D0000000003034C00002044000020F3
:102E20004C00002074010020AC00002018000000BD
:102E30000000000000000000000000000000000092
:102E40000000000000000000000000000000000082
:102E50000000000000000000000000000000000072
:102E60000020004000000000A42800000000000036
:102E70000000000000000000000000000000000052
:102E80000000000000000000000000000000000042
:102E9000782D0000182D0000702D0000202D00005E
:102EA000302D0000282D0000382D0000402D00009E
:102EB000482D0000502D0000582D0000602D00000E
:102EC000682D00000090D00300000000000000000A
:102ED00000000000000000000000000000000000F2
:042EE00000000000EE
:0400000500000201F4
:00000001FF
